:020000040000FA
:0400000071303A28F9
:08000800A000030EA100831209
:1000100005191028831601178312B23081002B288E
:1000200083160113831203140B190310A80DA90DD5
:10003000AA0DAB0DAC0DAC16FF302C02031D2B2806
:10004000FA302B02031D2B2831152A08AF0029088E
:10005000AE002808AD008B100B11210E8300A00EFE
:04006000200E090065
:0C007400203084008001840A6030040207
:10008000031C3C281230B0006A218316FF23900025
:10009000831283160C308505870183128501870141
:1000A000073099000030831691009F008312C830FA
:1000B00083168100831231309000003083168C004B
:1000C000831210308B00831600309B001C141A081A
:1000D0008312BC00831610309B001C141A08831274
:1000E000BD0083162F309B001C141A088312C30016
:1000F0008321831620309B001C141A088312C2002F
:100100000130C2080319C20081018E018F010B1159
:100110008B100B108C018B179C2031199F204E21C6
:10012000B30B9A28031085190314B90DF030390266
:100130000319F72086218C28640032100800311141
:100140000130B7008B132030370783169B001C1437
:100150001A088312A4001030370783169B001C1462
:100160001A088312A300A6000230A6060030370743
:1001700083169B001C141A088312A200A7000130EA
:10018000A7068B17321CCA2822090339A200A3092B
:10019000A409A50924082F02031DF12823082E0213
:1001A000031DDF2822082D02031DF128013037022C
:1001B000031DDF283D18DF283D143E147D2126084D
:1001C0002E02031DF12827082D02031DF1280130FE
:1001D0003702031DF0283D1CF0283D103E148121FC
:1001E000F128B70A0230370203180800A2280130AC
:1001F000B600B300B400B500B70085018701B113A4
:100200009C20B30B1D29031085190314B90DF03080
:10021000390203194429B41F8501B41F8701B40BA7
:100220001D293708B6080319B60003191B29FF302A
:1002300085008700B6039630B400311D00293111C6
:10024000321C27292D090339AD00AE09AF092F1C37
:1002500000298E018F010C1C00290C102E1E002974
:100260008B1320303707BB002F08BA0057211030FE
:100270003707BB002E08BA00572100303707BB00F4
:100280002D08BA0057218B1785018701B70AB601DF
:1002900002303702031C0029832108003E1C08009D
:1002A0003E101030BB003D08BA00572108008B13E8
:1002B0003A0883161C159A003B089B0055309D0098
:1002C000AA309D009C1464009C1863291C118312A1
:1002D0008B170800FF30D4000230D5000C30D60058
:1002E000BA30D7003730D800DA30D9006F30DA00B2
:1002F000B830DB000230C10008000130BD00DD1461
:100300000800DD1008003D18DD1408005C18051613
:10031000DC1885165C190514DC1985145C1A871421
:10032000DC1A07155C1B0714DC1B87165D18071603
:10033000DD1887155C1C0512DC1C85125C1D051080
:10034000DC1D85105C1E8710DC1E07115C1F07106A
:10035000DC1F87125D1C0712DD1C87118F08031933
:1003600008008F01C10B08004208C1005408DE00DC
:10037000FF22D4005508DE00FF22D5005608DE001B
:10038000541CFF22D6005708DE00D41CFF22D700E1
:100390005808DE00541DFF22D8005908DE00D41D85
:1003A000FF22D9005A08DE00541EFF22DA005B0843
:1003B000DE00D41EFF22DB005C08C6005D08C7001B
:1003C000CA0BF8295408CA008B13831640309B00CF
:1003D0001C141A0883125405031D5C148316503034
:1003E0009B001C141A0883125405031D5C108B1704
:1003F000CB0B102A5508CB008B13831641309B0082
:100400001C141A0883125505031DDC148316513081
:100410009B001C141A0883125505031DDC108B1752
:10042000CC0B282A5608CC008B13831642309B0035
:100430001C141A0883125605031D5C1583165230CE
:100440009B001C141A0883125605031D5C118B17A0
:10045000CD0B402A5708CD008B13831643309B00E9
:100460001C141A0883125705031DDC15831653301C
:100470009B001C141A0883125705031DDC118B17EF
:10048000CE0B582A5808CE008B13831644309B009D
:100490001C141A0883125805031D5C168316543069
:1004A0009B001C141A0883125805031D5C128B173D
:1004B000CF0B702A5908CF008B13831645309B0051
:1004C0001C141A0883125905031DDC1683165530B7
:1004D0009B001C141A0883125905031DDC128B178C
:1004E000D00B882A5A08D0008B13831646309B0005
:1004F0001C141A0883125A05031D5C178316563004
:100500009B001C141A0883125A05031D5C138B17D9
:10051000D10BA02A5B08D1008B13831647309B00B8
:100520001C141A0883125B05031DDC178316573051
:100530009B001C141A0883125B05031DDC138B1728
:10054000D20BB82A5608D2008B13831648309B0072
:100550001C141A0883125505031D5D1483165830A8
:100560009B001C141A0883125705031D5D108B177E
:10057000C4015C18C40ADC18C40A5C19C40ADC197A
:10058000C40A5C1AC40ADC1AC40A5C1BC40ADC1B59
:10059000C40A5D18C40AC5014618C50AC618C50AAA
:1005A0004619C50AC619C50A461AC50AC61AC50A91
:1005B000461BC50AC61BC50A4718C50A3D1CF62AB4
:1005C000430845020318ED2A4508440203180800B1
:1005D0004608DC004708DD00080043084402031811
:1005E00008004608DC004708DD0008004408450212
:1005F000031808004608DC004708DD000800C001B9
:10060000DE080319DE035E184014DE1A40144008A9
:10061000C0015E1C4014DE1E4014C005C00C5E0C00
:020620000800D0
:084000000E000300040008009B
:02400E00CC01E3
:10420000010078007A007C007E007B0079007F004E
:104210007D007A0078007E007C00FF00FF00FF0038
:104220000000F200F600FA00FE00F200F600FA00CC
:10423000FE00F200F600FA00FE00FF00FF00FF00A3
:10424000100005000500050005000900090009002F
:1042500009000D000D000D000D00FF00FF0005001E
:10426000FF00FF00FF00FF00FF00FF00FF00FF0056
:10427000FF00FF00FF00FF00FF00FF00FF00FF0046
:104280000800800002000800040010000400200064
:1042900004000200FF00FF00FF00FF00FF00FF001E
:1042A00001000100010004000800040010000400E7
:1042B00080000400FF00FF00FF00FF00FF00FF0080
:1042C000FF00FF00FF00FF00FF00FF00FF00FF00F6
:1042D000FF00FF00FF00FF00FF00FF00FF00FF00E6
:1042E000FF00FF00FF00FF00FF00FF00FF00FF00D6
:1042F000FF00FF00FF00FF00FF00FF00FF00DD00E8
:00000001FF
